:100C000012010002000000400E0B0A0D010001025B
:100C100000010A06000200000040010009022E0047
:100C200001010080320904000004FF0000000705F4
:100C30000202000200070504020002000705860206
:100C40000002000705880200020009022E000101CF
:100C50000080320904000004FF00000007050202C2
:100C6000400000070504024000000705860240001E
:100C70000007058802400000040309041203420033
:100C8000650072006B0065006C00650079002C0344
:100C90004200650072006B0065006C006500790021
:100CA0002000440041005100200042006F0061001C
:0C0CB000720064002000300031000000E1
:03004300020D00AB
:03005300020D009B
:100D0000020BE600020FAF00020F9900020F8100F4
:100D1000020EA000020CBC000210300002103100D4
:100D200002103200021033000210340002103500AD
:100D3000021036000210370002103800021039008D
:100D400002103A000210310002103B0002103C0079
:100D500002103D0002103E0002103F000210400051
:100D60000210410002103100021031000210310067
:100D7000021042000210430002104400021045001D
:100D800002104600021047000210480002104900FD
:100D900002104A0002104B0002104C0002104D00DD
:100DA00002104E0002104F000210500002105100BD
:080DB000021052000210530072
:0A10060000010202030304040505C3
:100A7B00E4F513F512F511F510C203C200C202C260
:100A8B00011210207E0C7F008E238F24752B0C758A
:100A9B002C1275210C75221C75290C752A4A752D83
:100AAB000C752E78EE54C07002617F7514007515AD
:100ABB00808E168F17C374BA9FFF740C9ECF2402BF
:100ACB00CF3400FEE48F0F8E0EF50DF50CF50BF504
:100ADB000AF509F508AF0FAE0EAD0DAC0CAB0BAABA
:100AEB000AA909A808C3120FE95037E517250BF51A
:100AFB0082E516350AF583E0FFE515250BF582E552
:100B0B0014350AF583EFF0E4FAF9F8E50B2401F557
:100B1B000BEA350AF50AE93509F509E83508F50850
:100B2B0080B385142385152474002480FF740C3442
:100B3B00FFFEC3E52C9FF52CE52B9EF52BC3E5267D
:100B4B009FF526E5259EF525C3E5289FF528E52786
:100B5B009EF527C3E5229FF522E5219EF521C3E5EE
:100B6B002A9FF52AE5299EF529C3E52E9FF52EE54B
:100B7B002D9EF52DD2E843D82090E668E04409F08D
:100B8B0090E65CE0443DF0D2AF90E680E020E105DA
:100B9B00D204120ED690E680E054F7F0538EF8C2D2
:100BAB0003120CFF300105120800C2013003F212D0
:100BBB000CFD50EDC203120F5C20001690E682E094
:100BCB0030E704E020E1EF90E682E030E604E0203D
:0A0BDB00E0E4120F0512102480C799
:010BE50022ED
:020BFE00D32200
:1008000090E6B9E0B40C004002416790081125E081
:100810007301C72162416721F241674167012941A4
:100820006701C201BD01B301B81210264002417335
:1008300090E6BBE024FE603414604924FD6013148C
:10084000603624067064E52390E6B3F0E524A3F057
:100850004173120BFE500CE52B90E6B3F0E52CA390
:10086000F0417390E6A0E04401F04173E52590E685
:10087000B3F0E526A3F04173E52790E6B3F0E52851
:10088000A3F0417390E6BAE0FF120F31AA06A90760
:100890007B01EA494B600AEE90E6B3F0EFA3F0412A
:1008A0007390E6A0E04401F0417390E6A0E04401BB
:1008B000F04173120FD741731210184173121010C8
:1008C0004173120FC541731210284002417390E624
:1008D000B8E0247F60251460332402707CA200E419
:1008E00033FF25E0FFA202E4334F90E740F0E4A39A
:1008F000F090E68AF0A37402F04173E490E740F0D0
:10090000A3F090E68AF0A37402F0417390E6BCE095
:10091000547EFF7E00E0D3948040067C007D018001
:10092000047C007D00EC4EFEED4F2406F582741031
:100930003EF583E493FF3395E0FEEF24A1FFEE3410
:10094000E68F82F583E0540190E740F0E4A3F09055
:10095000E68AF0A37402F0417390E6A0E04401F04F
:10096000417312102A4002417390E6B8E024FE6001
:100970001A24026002417390E6BAE0B40104C20096
:10098000417390E6A0E04401F0417390E6BAE07054
:100990005890E6BCE0547EFF7E00E0D39480400691
:1009A0007C007D0180047C007D00EC4EFEED4F2438
:1009B00006F58274103EF583E493FF3395E0FEEF75
:1009C00024A1FFEE34E68F82F583E054FEF090E63A
:1009D000BCE05480FF131313541FFFE0540F2F90FB
:1009E000E683F0E04420F0417390E6A0E04401F09B
:1009F000417312102C507C90E6B8E024FE60202455
:100A000002705B90E6BAE0B40104D200806590E623
:100A1000BAE06402605D90E6A0E04401F08054908A
:100A2000E6BCE0547EFF7E00E0D3948040067C006C
:100A30007D0180047C007D00EC4EFEED4F2406F528
:100A40008274103EF583E493FF3395E0FEEF24A11A
:100A5000FFEE34E68F82F583E04401F0801590E6E6
:100A6000A0E04401F0800C12102E500790E6A0E0A8
:0A0A70004401F090E6A0E04480F09D
:010A7A002259
:03003300020CF9C3
:040CF90053D8EF32AB
:100DB80090E6017443F000000090E6707440F00083
:100DC800000090E602748EF000000090E60374DCE8
:100DD800F0000000E490E609F000000090E60B74D3
:100DE80003F000000090E61274A2F000000090E604
:100DF8001474E0F000000090E6137420F000000086
:100E080090E615F000000090E6047480F000000001
:100E18007402F00000007408F0000000E4F0000024
:100E28000090E6497482F0000000F000000090E6AF
:100E3800187411F000000090E61A740DF00000001C
:100E480090E6247402F0000000E490E625F000002B
:020E5800002276
:04102000120DB822D3
:010CFF0022D2
:020CFD00D32200
:02102400D322D5
:02102600D322D3
:0810100090E6BAE0F51BD322C3
:100FC50090E740E51BF0E490E68AF090E68B04F0AC
:020FD500D32225
:0810180090E6BAE0F51AD322BC
:100FD70090E740E51AF0E490E68AF090E68B04F09B
:020FE700D32213
:02102800D322D1
:02102A00D322CF
:02102C00D322CD
:02102E00D322CB
:100BE600C0E0C083C082D2015391EF90E65D7401EC
:080BF600F0D082D083D0E03280
:100F9900C0E0C083C0825391EF90E65D7404F0D045
:060FA90082D083D0E0328B
:100FAF00C0E0C083C0825391EF90E65D7402F0D031
:060FBF0082D083D0E03275
:100EA000C0E0C083C082852925852A2685268285C3
:100EB0002583A37402F08521278522288528828531
:100EC0002783A37407F05391EF90E65D7410F0D080
:060ED00082D083D0E03265
:100F8100C0E0C083C082D2035391EF90E65D740844
:080F9100F0D082D083D0E032E1
:100CBC00C0E0C083C08290E680E030E7208521252B
:100CCC00852226852682852583A37402F085292713
:100CDC00852A28852882852783A37407F05391EFF2
:0D0CEC0090E65D7420F0D082D083D0E0321D
:01103000328D
:01103100328C
:01103200328B
:01103300328A
:011034003289
:011035003288
:011036003287
:011037003286
:011038003285
:011039003284
:01103A003283
:01103B003282
:01103C003281
:01103D003280
:01103E00327F
:01103F00327E
:01104000327D
:01104100327C
:01104200327B
:01104300327A
:011044003279
:011045003278
:011046003277
:011047003276
:011048003275
:011049003274
:01104A003273
:01104B003272
:01104C003271
:01104D003270
:01104E00326F
:01104F00326E
:01105000326D
:01105100326C
:01105200326B
:01105300326A
:100F050090E682E030E004E020E60B90E682E030F7
:100F1500E119E030E71590E680E04401F07F147EAA
:0C0F250000120E5A90E680E054FEF0220C
:100ED60030040990E680E0440AF0800790E680E05E
:100EE6004408F07FDC7E05120E5A90E65D74FFF032
:0F0EF60090E65FF05391EF90E680E054F7F02222
:020F3100A9070E
:100F3300AE2DAF2E8F828E83A3E064037017AD01B5
:100F430019ED7001228F828E83E07C002FFDEC3E31
:080F5300FEAF0580DFE4FEFFA4
:010F5B002273
:100F5C0090E682E044C0F090E681F0438701000007
:040F6C00000000225F
:100E5A008E188F1990E600E054187012E5192401D3
:100E6A00FFE43518C313F518EF13F519801590E64A
:100E7A0000E05418FFBF100BE51925E0F519E51835
:100E8A0033F518E5191519AE18700215184E6005D4
:060E9A00120F7080EE2231
:100F70007400F58690FDA57C05A3E582458370F994
:010F8000224E
:03000000020FFAF2
:0C0FFA00787FE4F6D8FD75812E020A7B9A
:100FE900EB9FF5F0EA9E42F0E99D42F0E89C45F05E
:010FF90022D5
:00000001FF
